:020000040000FA
:0600000040EF1FF01200AA
:0600080004EF10F01200ED
:060018000CEF10F01200D5
:0620000040EF1FF012008A
:0620080084EF19F0120044
:062018008DEF19F012002B
:06202A000100B43E0000BD
:082030006000000069000000DF
:08203800D9CFE6FFE1CFD9FF8B
:10204000E652A09A6A6A686A706A010EE66EE66AEB
:10205000E66A710EE66E0F0EE66E06EC1FF00B6E72
:10206000050EE15E0B50160E6F6E9F0E6B6E7B0EB3
:10207000696EDF6ADF500B6E0C6A080E0B5C000E97
:102080000C5810E2DF50040DF3CFE9FFF4CFEAFF64
:10209000000EE926040EEA22EE6AEE6AEE6AEE6AA5
:1020A000DF2AE8D76D8C6E6A6D986D9C68A607D0A4
:1020B00068960001DC6BE16BE26BE36BF7D7000124
:1020C000010EF36FF46FF56BF66BE96BDF6A020ECE
:1020D000DF5C26E2EA6ADF34FE0BEA36E96ED40EF4
:1020E000E926000EEA22EE6AED6AEA6ADF34FE0BA8
:1020F000EA36E96ED00EE926000EEA22EE6AED6AB3
:10210000DF50EA6AED0FE96E000EEA22EF6ADF5057
:10211000EA6AEF0FE96E000EEA22EF6ADF2AD7D7EC
:102120000001080ED46F040ED56F160E706E0401F8
:10213000200E026F040E036F080E016F840E006FF5
:102140000001CA6BC96BE552E552E7CFD9FF120017
:10215000D9CFE6FFE1CFD9FFE6520001C95116E120
:1021600006D06D6A696A0001C96BA19AB6D06D6A22
:10217000696A160E6F6E9F0E6B6E7B0E696E6DB682
:1021800002D06D86FCD70001010EC96FC90508E1B8
:102190006DBA06D0686A696A69806988020EC96F7B
:1021A0006850040B06E06950040B03E06894AEEC41
:1021B00016F06DA202D0A19A90D06850010B08E0F1
:1021C0006950010B05E038DF0001040EC96F68900B
:1021D0006850100B06E06950100B03E099EC16F004
:1021E000689868AC12D069AC0FD0010EE66EE66A52
:1021F000000EE66EE66A730EE66EE66A85EC1DF08A
:102200000B6E060EE15E0B50689C6850200B05E0DB
:102210006950200B02E080EC16F06850020B13E0CE
:102220006950020B10E0010EE66EE66A000EE66EE3
:10223000E66AE6687F0EE66E85EC1DF00B6E060E14
:10224000E15E0B506A6A040E0001E76EC919E8AE40
:1022500002D0E73402D0E750C95D02E2A19A3DD036
:1022600069A63AD0DF6A040EDF5C36E268A631D098
:102270006CCFEAF00001EA51780BE842E842E8420C
:10228000EB6F6896EAB508D0EB51EA6AEF0FE96E9A
:10229000000EEA22EF7007D0EB51EA6AED0FE96E0B
:1022A000000EEA22EF70EB5103E1C5EC16F010D0FE
:1022B000000EE66EE66AEA0EE66E000EE66E720E3E
:1022C000E66EE66A85EC1DF00B6E060EE15E0B50C5
:1022D00001D002D0DF2AC7D7A19AE552E552E7CF55
:1022E000D9FF1200D9CFE6FFE1CFD9FF020EE126D8
:1022F000FD0EDBA407D0E66AFE0EDBCFE6FF05DAB3
:10230000E552E552FD0EDBA208D0010EE66EFE0E90
:10231000DBCFE6FFFAD9E552E552FE0EDB500C6A40
:10232000700F0B6E0F0E0C220BC0DEFF0CC0DDFF1A
:10233000DECFE9FFDDCFEAFFFD0EDBCFEFFF020EC0
:10234000E15C02E2E16AE552E16EE552E7CFD9FFD6
:102350001200D9CFE6FFE1CFD9FF020EE126FD0E34
:10236000DB500FE0FE0EEA6ADB34FE0BEA36E96E64
:10237000D40EE926000EEA22EECFDEFFEDCFDDFF20
:102380000ED0FE0EEA6ADB34FE0BEA36E96ED00EA2
:10239000E926000EEA22EECFDEFFEDCFDDFFD9CF3A
:1023A000E9FFDACFEAFFEE50ED1003E1F36AF46AD9
:1023B00049D0DECFE9FFDDCFEAFF020EE926000EAD
:1023C000EA22FB0EDBCFEEFFFC0EDBCFEDFFDECF14
:1023D000E9FFDDCFEAFFEE52FA0EDBCFEFFF400E52
:1023E0000B6EDECFE9FFDDCFEAFF0B50EF16880E54
:1023F0000B6EDECFE9FFDDCFEAFF0B50EF12FD0ED3
:10240000DB500CE0FE0EEA6ADB34FE0BEA36E96EC6
:10241000D40EE926000EEA22EF740BD0FE0EEA6A13
:10242000DB34FE0BEA36E96ED00EE926000EEA2216
:10243000EF74DECF0BF0DDCF0CF00BC0F3FF0CC060
:10244000F4FF00D0020EE15C02E2E16AE552E16EC7
:10245000E552E7CFD9FF1200D9CFE6FFE1CFD9FF90
:10246000020EE126FE0EDB5020E1CEC0E9FFCFC018
:10247000EAFFEE52080EEF6ECEC0E9FFCFC0EAFFD2
:10248000020EE926000EEA22200EEE6E040EED6E1C
:10249000CEC0E9FFCFC0EAFF8C0EEF6ED4C0E9FFDB
:1024A000D5C0EAFF840EEF6E3DD0FD0EDB50E82470
:1024B0000D6EFE0EDB50040DF3500D24040DF3CF12
:1024C0000BF0F4CF0CF0000E0B26040E0C220BC008
:1024D000DEFF0CC0DDFF840E0B6EDECFE9FFDDCF2B
:1024E000EAFF0B50EF12FD0EDB50E8240D6EFE0EDE
:1024F000DB50040DF3500D24010F040DF3CF0BF04E
:10250000F4CF0CF0000E0B26040E0C220BC0DEFFE5
:102510000CC0DDFF840E0B6EDECFE9FFDDCFEAFFDE
:102520000B50EF12020EE15C02E2E16AE552E16E4D
:10253000E552E7CFD9FF1200D9CFE6FFE1CFD9FFAF
:102540006DA84ED0FE0EEA6ADB34FE0BEA36E96E69
:10255000D40EE926000EEA22EE50EFCFEAFFE96E34
:10256000400EEE16EE6AEE6AEE6AFE0EEA6ADB34A2
:10257000FE0BEA36E96ED40EE926000EEA22EE5092
:10258000EFCFEAFFE96EEE7CFE0EEA6ADB34FE0B6B
:10259000EA36E96ED40EE926000EEA22EF74400E08
:1025A0000B6EFE0EEA6ADB34FE0BEA36E96ED40EE1
:1025B000E926000EEA22EE50EFCFEAFFE96E0B505B
:1025C000EF16FE0EEA6ADB34FE0BEA36E96ED40E35
:1025D000E926000EEA22EE50EFCFEAFFE96EEF7C2B
:1025E000E552E7CFD9FF12000001F3514DE1010E92
:1025F000F36FF45149E1010EF46F020ED95D0DE164
:10260000D4C0E9FFD5C0EAFFEE52EF6AD4C0E9FFBB
:10261000D5C0EAFFC80EEF6E37D0D90535E1EC6BB7
:10262000CCC0E9FFCDC0EAFFEE52080EEF6ECCC081
:10263000E9FFCDC0EAFF020EE926000EEA22200ED5
:10264000EE6E040EED6ECCC0E9FFCDC0EAFF840E45
:10265000EF6E010EEC6FCEC0E9FFCFC0EAFFEE5285
:10266000080EEF6ECEC0E9FFCFC0EAFF020EE926EA
:10267000000EEA22200EEE6E040EED6ECEC0E9FFD3
:10268000CFC0EAFF800EEF6E12000001F56BF66B13
:10269000020ED95D1AE1CEC0E9FFCFC0EAFFEE52CB
:1026A000080EEF6ECEC0E9FFCFC0EAFF020EE926AA
:1026B000000EEA22280EEE6E040EED6ECEC0E9FF8B
:1026C000CFC0EAFFC80EEF6E1FD0DD510401265DBA
:1026D0000001DE510401275904E226C4DDF027C4BD
:1026E000DEF0D1D8D4C0E9FFD5C0EAFF020EE9265A
:1026F000000EEA22280EEE6E040EED6ED4C0E9FF45
:10270000D5C0EAFFC80EEF6E1200D9CFE6FFE1CFC9
:10271000D9FF020EE126000EDE6E040EDD6EFD0E08
:10272000DB50E8240D6EFE0EDB50040DF3500D243B
:10273000040DF3CF0BF0F4CF0CF0D9CFE9FFDACFD3
:10274000EAFF0B50EE260C50ED22DECFE9FFDDCF85
:10275000EAFFEF9EFD0EDB500FE1FE0EEA6ADB346E
:10276000FE0BEA36E96ED00EE926000EEA22DECF35
:10277000EEFFDDCFEDFF0ED0FE0EEA6ADB34FE0B7E
:10278000EA36E96ED40EE926000EEA22DECFEEFF2D
:10279000DDCFEDFFDECFE9FFDDCFEAFFEF9CDECF3F
:1027A000E9FFDDCFEAFF040EE926000EEA22EF8CF6
:1027B000020EE15C02E2E16AE552E16EE552E7CF2A
:1027C000D9FF12006D980001DCBF2BD0E1AF09D01A
:1027D000020ED96FF65101E158DF0001F46BF36B83
:1027E0001FD0CEC0E9FFCFC0EAFFEE52080EEF6E59
:1027F000CEC0E9FFCFC0EAFF020EE926000EEA22B2
:10280000200EEE6E040EED6ECEC0E9FFCFC0EAFFE3
:102810008C0EEF6ED4C0E9FFD5C0EAFF840EEF6ED8
:1028200031D0040120AF0DD00001010ED96FF55158
:1028300001E12BDF0001F46BF36BF25101E1D4DE17
:1028400021D00001020ED96FCEC0E9FFCFC0EAFF50
:10285000EE52080EEF6ECEC0E9FFCFC0EAFF020EC7
:10286000E926000EEA22200EEE6E040EED6ECEC0BA
:10287000E9FFCFC0EAFF840EEF6EF46BF36BF25109
:1028800001E1B2DE1200D9CFE6FFE1CFD9FFE65277
:10289000080EDF6E0001DD5D000EDE590BE2DDC0CB
:1028A000DFFFD85103E1010ED86F04D0D80502E153
:1028B000020ED86FDF500B6E0C6A0B50DD5DDD6FC2
:1028C0000C50DE59DE6FD4C0E9FFD5C0EAFFEE52EE
:1028D000DFCFEFFF280EE66F040EE76FDCB119D0F3
:1028E000DF5016E0DAC0F6FFDBC0F7FFDA2B000E90
:1028F000DB230800F550E66EE6C0E9FFE7C0EAFF1B
:10290000E62B000EE723E552E750EF6EDF06E8D72F
:1029100017D0DF5015E0DAC0E9FFDBC0EAFFDA2BA1
:10292000000EDB23EF50E66EE6C0E9FFE7C0EAFFEA
:10293000E62B000EE723E552E750EF6EDF06E9D7FE
:10294000E552E552E7CFD9FF1200D9CFE6FFE1CF3C
:10295000D9FF020EE126CCC0E9FFCDC0EAFFEE525E
:10296000EFCFDFFFDFCF0BF00B500001E25D000E79
:10297000E35902E2E2C0DFFFDF500B6E0C6A0B503E
:10298000E25DE26F0C50E359E36F010EDB6ADF504A
:10299000F36E010EDBCFF4FFF350F45C16E2010E90
:1029A000DB50EA6A280FE96E040EEA22EF50E66E69
:1029B000DFC0E9FFE0C0EAFFDF2B000EE023E552B5
:1029C000E750EF6E010EDB2AE2D7000ED880E25509
:1029D000000EE35528E2CEC0E9FFCFC0EAFFEE5279
:1029E000080EEF6ECEC0E9FFCFC0EAFF020EE92667
:1029F000000EEA22280EEE6E040EED6ECCC0E9FF4A
:102A0000CDC0EAFFEF50400B07E1CEC0E9FFCFC0D9
:102A1000EAFFC80EEF6E06D0CEC0E9FFCFC0EAFFD6
:102A2000880EEF6E28D0CEC0E9FFCFC0EAFFEE528D
:102A3000080EEF6ECEC0E9FFCFC0EAFF020EE92616
:102A4000000EEA22200EEE6E040EED6ECEC0E9FFFF
:102A5000CFC0EAFF840EEF6EE451E51107E005D028
:102A6000E5C0FAFF0001E451F96EFADF0001E19FD1
:102A7000F25101E1B9DD020EE15C02E2E16AE552E8
:102A8000E16EE552E7CFD9FF1200D9CFE6FFE1CFE3
:102A9000D9FFE6520001DC8F010EE66EE66AE66AB7
:102AA000710EE66E0F0EE66E06EC1FF00B6E050E55
:102AB000E15E0B50200EE66EE66AE66A000EE66EF8
:102AC000040EE66E06EC1FF00B6E050EE15E0B5079
:102AD0006D8CDF6A020EDF5C10E2DF50EA6AED0FF8
:102AE000E96E000EEA22EF6ADF50EA6AEF0FE96E44
:102AF000000EEA22EF6ADF2AEDD7010EE66EE66AE3
:102B0000E66ACB0EE66E000EE66E06EC1FF00B6E6C
:102B1000050EE15E0B506D9C0001080ED46F040E93
:102B2000D56F000ECC6F040ECD6FCCC0CEF0CDC0F3
:102B3000CFF022C4CAF0CA5103E1100EC96F13D0FE
:102B4000010EE66EE66ACA0EE66E000EE66E010E35
:102B5000E66EE66A85EC1DF00B6E060EE15E0B502C
:102B60000001200EC96FE552E552E7CFD9FF1200F0
:102B7000800E0401205D5BE10001C00EDC6F0401EA
:102B80002351030A34E0010A0EE0030A03E00001C6
:102B9000DC6B4DD00001A00EDA6F3B0EDB6F120E26
:102BA000DD6FDE6B44D02251F66EF76AD890F636B0
:102BB000F736410EF6263C0EF7220900F5CFDAF083
:102BC0000A00F5CFDBF0020E0001F76ADA25F66E97
:102BD000DB51F7220800F5CFDDF0030EF76ADA25A6
:102BE000F66EDB51F7220800F5CFDEF020D0030EA1
:102BF000225D1AE22251F66EF76AD890F636F73661
:102C0000430EF6263C0EF7220900F5CFDAF00A0053
:102C1000F5CFDBF0DAC0F6FFDBC0F7FF0800F550B8
:102C20000001DD6FDE6B02D00001DC6B00D0120012
:102C3000D9CFE6FFE1CFD9FF020EE1260401286BD0
:102C4000296B20511F0B020A12E0030A0DE0010A52
:102C500001E042D00001DC8F040128810001E80579
:102C600002E10401288338D00001DC8F35D0000157
:102C7000DC8F040124BF10D024510F0BE96EEA6AE7
:102C8000D890E936EA36D00EE926000EEA22EECFD9
:102C9000DEFFEDCFDDFF0FD024510F0BE96EEA6AA6
:102CA000D890E936EA36D40EE926000EEA22EECFB5
:102CB000DEFFEDCFDDFFDECFE9FFDDCFEAFFEF5036
:102CC000800B09E0DECFE9FFDDCFEAFFEF50040B18
:102CD00002E0010E286F00D00001DCAF07D0280E03
:102CE000DA6F040EDB6FDC81020EDD6F020EE15C39
:102CF00002E2E16AE552E16EE552E7CFD9FF120048
:102D000070A015D0CCC0E9FFCDC0EAFFEF5080081D
:102D10000DE1D4C0E9FFD5C0EAFFEF50840806E119
:102D2000CCC0E9FFCDC0EAFF8C0EEF6E7090689AC0
:102D30001200698468986D820001010EE96F000E2F
:102D4000E66EE66AE66EE66A750EE66EE66A85ECA3
:102D50001DF00B6E060EE15E0B5012000001E96BD8
:102D6000000EE66EE66AE66EE66A740EE66EE66AE7
:102D700085EC1DF00B6E060EE15E0B506D926994B2
:102D800068A402D06894FCD71200D9CFE6FFE1CF47
:102D9000D9FFE652FD0E0001EA1553E17E0EEA1559
:102DA000E8407F0B040DF3CFCCF0F4CFCDF0000E54
:102DB000CC27040ECD23CCC0CEF0CDC0CFF0CE7545
:102DC000CCC0E9FFCDC0EAFFEF503C0BE842E8423F
:102DD0000D0835E1DF6A080EDF5C23E2CCC0E9FFB5
:102DE000CDC0EAFF020EE926000EEA22EE50EFCF38
:102DF000EAFFE96EEF50E66EDF50EA6A200FE96EF7
:102E0000040EEA22E552E750EF6ECCC0E9FFCDC0D8
:102E1000EAFF020EE926000EEA22EE2AEF22DF2A5E
:102E2000DAD7CCC0E9FFCDC0EAFF020EE926000EDA
:102E3000EA22200EEE6E040EED6E0DD801D03AD8C7
:102E400005D0FD0EEA15040801E159D8E552E55216
:102E5000E7CFD9FF12000001D86BF26BF56BF66B70
:102E6000EC6BD96BD4C0E9FFD5C0EAFFEF9ED475F7
:102E7000D4C0E9FFD5C0EAFFEF9ED475CEC0E9FF0C
:102E8000CFC0EAFFEF9EDC6BDD6BDE6BE16BE26BCC
:102E9000E36B8FD8000EE66EE66AE66EE66A030E16
:102EA000E66EE66A85EC1DF00B6E060EE15E0B50D9
:102EB000E2EF13F0020E0001D95D02E146DD1ED003
:102EC000D96BEC511AE1CEC0E9FFCFC0EAFFEE5258
:102ED000080EEF6ECEC0E9FFCFC0EAFF020EE92672
:102EE000000EEA22200EEE6E040EED6ECEC0E9FF5B
:102EF000CFC0EAFF8C0EEF6E01D0EC6B1200D9CF81
:102F0000E6FFE1CFD9FFE652D4C0E9FFD5C0EAFF22
:102F1000EF50400B01E0010EDF6E0001D475080E8A
:102F2000C95D09E122C46EFF6E5003E0100EC96F47
:102F300002D0040EC96FD90528E1D4C0E9FFD5C07D
:102F4000EAFF020EE926000EEA22280EEE6E040EBB
:102F5000ED6E99DC020E0001D85D07E1D4C0E9FFF7
:102F6000D5C0EAFF840EEF6E0FD0DF5007E1D4C06A
:102F7000E9FFD5C0EAFFC80EEF6E06D0D4C0E9FF66
:102F8000D5C0EAFF880EEF6E0FD0E1AF0CD0E45150
:102F9000E51107E005D0E5C0FAFF0001E451F96E44
:102FA000FADF0001E19FD96BE552E552E7CFD9FF87
:102FB000120004012051600BE842E842E842E84276
:102FC000E842000901E058D021510C0A54E00B0AF4
:102FD00043E00C0A35E0010A26E00B0A22E0020A6F
:102FE00020E0030A1CE0080A10E0010A0CE00F0AC6
:102FF00008E0030A01E03FD00001DC8F080EC96F32
:103000003BD0B6DD39D041DD37D00001CA0EDA6FD2
:10301000000EDB6FDC81010EDD6FDC8F2DD008DE52
:103020002BD02BD829D024510001DA6FDB6BCB0ECB
:10303000DA27000EDB23DC81010EDD6FDC8F1CD074
:103040000001DC8F04012451EA6ACB0FE96E000E07
:10305000EA2222C4EFFF10D0000EE66EE66AE66EAA
:10306000E66A020EE66EE66A85EC1DF00B6E060E51
:10307000E15E0B5001D000D01200D9CFE6FFE1CFC6
:10308000D9FF050EE1260401220510E120511F0B96
:1030900000090CE10001DC8F030E0401215D04E155
:1030A0000001010EE86F02D00001E86B040122511B
:1030B00001E020D120511F0B020801E01BD1245157
:1030C0000F0B000901E116D124510F0B010801E299
:1030D00011D1200E0001C95D01E00CD1DC8F04018B
:1030E00024BF1AD024510F0BE96EEA6AD890E93652
:1030F000EA36D00EE926000EEA22EECFDEFFEDCF53
:10310000DDFF24510F0BEA6AEF0FE96E000EEA2291
:10311000020EEFCFDBFF19D024510F0BE96EEA6AE4
:10312000D890E936EA36D40EE926000EEA22EECF30
:10313000DEFFEDCFDDFF24510F0BEA6AED0FE96EE4
:10314000000EEA22020EEFCFDBFFD950020FE96E2C
:10315000DACFEAFFEF50010B03E1000EDF9401D05C
:10316000DF8424BF10D024510F0BE96EEA6AD89097
:10317000E936EA36D00EE926000EEA22DECFEEFF6F
:10318000DDCFEDFF0FD024510F0BE96EEA6AD89026
:10319000E936EA36D40EE926000EEA22DECFEEFF4B
:1031A000DDCFEDFF030E215D23E1DECFE9FFDDCFB3
:1031B000EAFFEF50800B13E024BF09D024510F0B1E
:1031C000EA6AEF0FE96E000EEA22EF8208D024517E
:1031D0000F0BEA6AED0FE96E000EEA22EF82840E11
:1031E0000B6EDECFE9FFDDCFEAFF0B50EF1282D08E
:1031F000DF74DECFE9FFDDCFEAFFEF50800B1BE08D
:10320000DECFE9FFDDCFEAFFEF9EDECFE9FFDDCFC6
:10321000EAFFEF8C020EE66EE66ADECFE6FFDDCF58
:10322000E6FF050EE66EE66A85EC1DF00B6E060EF7
:10323000E15E0B5005D0DECFE9FFDDCFEAFFEF8C7A
:10324000DF74D950020FE96EDACFEAFFEF50020BBC
:1032500007E1DECFE9FFDDCFEAFFEF50800B2DE085
:10326000040124BF09D024510F0BEA6AEF0FE96E65
:10327000000EEA22EF9208D024510F0BEA6AED0FFC
:10328000E96E000EEA22EF923B0E0B6EDECFE9FFF5
:10329000DDCFEAFF0B50EF16020EE66EE66ADECFD8
:1032A000E6FFDDCFE6FF050EE66EE66A85EC1DF073
:1032B0000B6E060EE15E0B5008D03B0E0B6EDECFA0
:1032C000E9FFDDCFEAFF0B50EF16040124510F0B8D
:1032D0000C6A700F0B6E0F0E0C22030E0BC0DBFF7F
:1032E000040E0CC0DBFF030EDBCFE9FF040EDBCFC7
:1032F000EAFFEF90050EE15C02E2E16AE552E16E61
:08330000E552E7CFD9FF1200EE
:08330800DACFE4FFE2CFDAFFA7
:10331000E652E552E5CFDAFF1100D8CFE4FFE0CF67
:10332000E4FFE46EDACFE4FFE2CFDAFFE652E552E3
:10333000E5CFDAFFE550E5CFE0FFE5CFD8FF10009D
:1033400005D8A8EC10F017D8FCD712000F0EC11248
:1033500002D81CEF10F092689368F80E946E806AA1
:10336000816A826A896A8A6A8B6A0101086B096BC1
:103370000A6B0B6B1200200E0001E76EC919E8AE54
:1033800002D0E73402D0E750C95D03E36D50020B71
:1033900001E001D06BD81200D9CFE6FFE1CFD9FF11
:1033A000FD0EDB5052E101010F6B106B0E6BF29EB4
:1033B0000D6B080EE76E0D19E8AE02D0E73402D0AF
:1033C000E7500D5D31E20A0EE66E4EEC1FF0E5525D
:1033D0009392FE0EDB50010BE8B0948EE8A0949E11
:1033E000FE0EDB407F0BE76EFE0EE7CFDBFF0A0E23
:1033F000E66E4EEC1FF0E55201010F417F0B0F6F9F
:1034000010417F0B106F8150010B800DF3500F1195
:103410000F6F8050040B01E0010E800DF35010116E
:10342000106F93820D2BC5D781A60ED00E2B640E84
:10343000E76E0E19E8AE02D00E3503D0E750D88003
:103440000E5501E201D0F0D7F28EFD0EDB0403E150
:1034500001010F5107D0FD0EDB50020803E101010D
:10346000105100D0E552E7CFD9FF1200D9CFE6FFC7
:10347000E1CFD9FF040EE126DF6A93949292DFCF69
:103480000BF000016051E76E0B18E8AE02D0E73494
:1034900002D0E7500B5C5DE2E66ADFCFE9FFEA6A43
:1034A000E9BEEA68610EE926000EEA22EF50E66EF8
:1034B00073DFE552E552010EE66EDFCFE9FFEA6AFF
:1034C000E9BEEA68610EE926000EEA22EF50E66ED8
:1034D00063DFE552E552E66EDFCFE9FFEA6AE9BE57
:1034E000EA68810EE926000EEA22E552E750EF6E07
:1034F000020EE66EDFCFE9FFEA6AE9BEEA68610E16
:10350000E926000EEA22EF50E66E46DFE552E5526C
:10351000E66EDFCFE9FFEA6AE9BEEA68A10EE926B6
:10352000000EEA22E552E750EF6E0F0E0001821501
:10353000E824030F606F020EDF5C09E15A0E835D21
:1035400006E093849282050E606FB7D201D0DF2A25
:1035500096D7938492828251410A01E005D084C0BB
:1035600011F185C012F100D0410EA25D03E0730E8F
:10357000A25D0CE1A4C017F1A5C018F1A6C019F115
:10358000A7C01AF1A8C01BF1A9C01CF10501006B6E
:103590000369080E046F056B01011151200B01E056
:1035A000010E040DF3CF0CF01151800B01E0010E60
:1035B000E8240B6E1251100B01E0010E0B240C24B9
:1035C000E76E020EE7CFDBFFDB500EE0020EDBCF33
:1035D0000BF0060EE76E0B18E8AE02D00B3403D0EA
:1035E000E750D8800B5401E268D21251020B01E07F
:1035F000010E080DF3CF0DF01251080B01E0010E82
:10360000040DF3CF0CF01251010BE8240B6E125194
:10361000040B01E0010E0B240C240D24E76E030EB5
:10362000E7CFDBFFDB5001E148D2020EDB50060A98
:103630001FE0030A19E0010A13E0070A0DE0010A7E
:1036400007E0030A01E017D00501810E026F15D0D3
:1036500005016D0E026F11D00501540E026F0DD0E1
:1036600005013F0E026F09D00501210E026F05D042
:103670000501026B02D005010269030EDB500F0A3F
:1036800047E0010A42E0030A3DE0010A38E0070A88
:1036900033E0010A2EE0030A29E0010A24E00F0AC0
:1036A0001FE0010A1AE0030A15E0010A10E0070A08
:1036B0000BE0010A06E0030A01E02DD0790E016F4C
:1036C0002CD08A0E016F29D0940E016F26D09A0E4D
:1036D000016F23D0A20E016F20D0A80E016F1DD064
:1036E000AF0E016F1AD0B20E016F17D0B50E016F79
:1036F00014D0B50E016F11D0B50E016F0ED0B90EFA
:10370000016F0BD0B90E016F08D0B90E016F05D053
:10371000B90E016F02D0016900D0010112BF13D0B0
:10372000640E0001E76EC219E8AE02D0E73402D0A1
:10373000E750C25D01E2C22B0F0EC25D04E1C56B12
:10374000010EC66FC46B010112AF1BD0000E000149
:10375000E76EC219E8AE02D0C23503D0E750D88078
:10376000C2550DE20F0EE76EC219E8AE02D0E73483
:1037700002D0E750C25D03E2010EC56FC46BC26B9D
:10378000C66B0001C50517E1640EE76EC419E8AE0B
:1037900002D0E73402D0E750C45D01E2C42B050E2D
:1037A000E76EC419E8AE02D0C43503D0E750D88024
:1037B000C45501E2C56B010111B113D0640E0001C3
:1037C000E76EC119E8AE02D0E73402D0E750C15D20
:1037D00001E2C12B0F0EC15D04E1C76B010EC86F82
:1037E000C36B010111A11BD0000E0001E76EC119CE
:1037F000E8AE02D0C13503D0E750D880C1550DE204
:103800000F0EE76EC119E8AE02D0E73402D0E750E0
:10381000C15D03E2010EC76FC36BC16BC86B0001D2
:10382000C70517E1640EE76EC319E8AE02D0E734AE
:1038300002D0E750C35D01E2C32B050EE76EC3194A
:10384000E8AE02D0C33503D0E750D880C35501E2BB
:10385000C76B01011751010BE81C0001C7110501DD
:103860000599E8B005890001C8515BE101011851D3
:10387000800B01E0010EE81C0001C6110501059353
:10388000E8B0058301011851400B01E0010EE81C6E
:103890000B6E1251400B01E0010EE81C0B100501EC
:1038A0000591E8B0058101011851200B01E0010EDE
:1038B000E81C0B6E1251200B01E0010EE81C0B10EE
:1038C00005010595E8B0058501011851100B01E0CF
:1038D000010EE81C0001C51105010597E8B0058738
:1038E000010117B905D005010491049304950497CB
:1038F000010117BB05D005010491048304950497C9
:10390000010117BD05D005010491049304850497B6
:10391000010117BF05D005010491048304850497B4
:103920001FD0C60505E10501049104930495049791
:10393000010112BB05D0050104910483049504978D
:10394000010112BD05D0050104910493048504977B
:103950000001C50505E10501049104830485049770
:1039600001011751080B01E0010EE81C0B6E11510B
:10397000080B01E0010EE81C0B100501059BE8B0E7
:10398000058B0A0EE66E20EC1FF0E552010108518E
:10399000091102E1000E08D008C1E9FF09C1EAFFE0
:1039A000EF50800B01E0010E000963E1010EDB6ABC
:1039B000DF6ADFCF0BF00C6A0BBE0C68060E0B5CE7
:1039C000000E0C581CE2DFCFE9FFEA6AE9BEEA68A4
:1039D000060EE926050EEA22EFCF0BF0DFCFE9FF56
:1039E000EA6AE9BEEA68000EE926050EEA22EF500F
:1039F0000B5C03E0DE52010EDD6EDF2ADAD7010E2A
:103A0000DB0413E1060EE66E000EE66E050EE66EB2
:103A1000010EE66EE66EA9EC11F00B6E050EE15E8E
:103A20000B50F3CF08F1F4CF09F1DF6ADFCF0BF0D1
:103A30000C6A0BBE0C68060E0B5C000E0C5819E2EB
:103A4000DFCFE9FFEA6AE9BEEA68000EE926050E63
:103A5000EA22EF50E66EDFCFE9FFEA6AE9BEEA68E4
:103A6000060EE926050EEA22E552E750EF6EDF2A40
:103A7000DDD701010A510B1102E1000E08D00AC185
:103A8000E9FF0BC1EAFFEF50800B01E0010E0009D6
:103A900013E1080EE66E140EE66E050EE66EE66A9B
:103AA000010EE66EA9EC11F00B6E050EE15E0B50F7
:103AB000F3CF0AF1F4CF0BF100D0040EE15C02E287
:103AC000E16AE552E16EE552E7CFD9FF120012003C
:103AD0001200120012004BEF1EF012001E0EE66ED6
:103AE000010EE66E72EC11F0E552E55212006D84A3
:103AF0000101080E1D6F070E1E6F1D07000E1E5BD5
:103B00001D511E11FAE16D941200D9CFE6FFE1CFED
:103B1000D9FFFD0EDBCF06F0FE0EDBCF07F0720EF5
:103B2000061801E1075033E0E868061802E17F0E4D
:103B300007182BE0740E061801E1075024E0750EFB
:103B4000061801E107501DE0730E061801E1075049
:103B500016E0030E061801E107500FE0020E0618EA
:103B600001E1075008E0010E061801E1075001E0ED
:103B700010D0B4DF0FD0B1DF0DD0ADDF0BD0A9DF97
:103B800009D0A5DF07D0A4DF05D0A4DF03D0000053
:103B900001D000D0010E00D0E552E7CFD9FF1200CE
:103BA00012011001FF040008E40A040000010102F0
:103BB000030109021900010100A0FA090400000133
:103BC00003000000070581030800140403090434FE
:103BD000034D006900630072006F006300680069B4
:103BE000007000200054006500630068006E006FE4
:103BF000006C006F0067007900200049006E0063D0
:103C0000002E002A0354004100490054004F005F79
:103C100000440045004E005300590041005F00433E
:103C2000004F004E005F0054003000310014035478
:103C300000430050005000320030003000310030AE
:103C400000B23BCB3BCF3B033C2D3C05010905A11A
:103C50000115002501350045017501950D0509196E
:103C600001290C81029503810105012507463B01CD
:103C7000750495016514093981426500950181013A
:103C800026FF0046FF000930093109320935750861
:053C900095048102C053
:0A3C9600040120511F0B010801E09A
:103CA00065D0245101E062D0060E215D22E123514E
:103CB000230A1EE0010A11E0030A01E01AD0000104
:103CC000CA050AE10001C40EDA6F3B0EDB6F090E74
:103CD000DD6FDE6BC00EDC6F0CD000014B0EDA6FB7
:103CE0003C0EDB6F4A0EDD6FDE6BC00EDC6F01D069
:103CF00000D004012051600BE842E842E842E8426B
:103D0000E842010801E032D021510B0A29E0080AFB
:103D10001CE0090A14E0080A07E00B0A04E0080A9C
:103D200001E024D023D022D00001F70EDA6F000E7C
:103D3000DB6F010EDD6FDE6BC10EDC6F17D0000193
:103D4000800EDC6F23C4F7F011D00001F80EDA6F9B
:103D5000000EDB6F010EDD6FDE6B810EDC6F06D0B7
:0E3D60000001800EDC6F22C4F8F000D01200CB
:023D6E002A0E1B
:103D7000F66E200EF76E000EF86E01010900F55088
:103D8000246F0900F550256F03E1246701D03DD071
:103D90000900F5501F6F0900F550206F0900F5501C
:103DA000216F09000900F550E96E0900F550EA6E2F
:103DB000090009000900F550226F0900F550236F32
:103DC00009000900F6CF26F1F7CF27F1F8CF28F147
:103DD0001FC1F6FF20C1F7FF21C1F8FF01012253E7
:103DE00002E1235307E00900F550EE6E2207F8E2E6
:103DF0002307F9D726C1F6FF27C1F7FF28C1F8FF2F
:0C3E000001012407000E255BBFD7120053
:043E0C00FE0EE3CFF4
:103E1000E9FFFF0EE3CFEAFFE9CFF3FFEACFF4FFBC
:103E2000FB0EE35003E1FC0EE35009E0FB0EE3065A
:103E300002E2FC0EE306FD0EE350EE6EF1D7120037
:103E4000FF0EE3500E6E480E01D04C0EE76EE72ECB
:103E5000FED7E76AE72EFED70E2EF7D70000120036
:103E6000000EF36E00EE00F0080E01D81200EA60BA
:103E700002D0EE6AFCD7F350E9601200EE6AFCD77C
:103E800013EE00F023EE00F0F86A0A9CB7EC1EF087
:0C3E900059EC1FF0A0EC19F0FBD7120059
:043E9C00FF0EE350E2
:103EA000E84E1200000000D000D000D0E82EFAD773
:023EB0001200FE
:023EB2001200FC
:0C3EB400050142000000000000000000BA
:103EC00000000000000000000000000000000000F2
:103ED00000000000000000000000000000000000E2
:103EE00000000000000000000000000000000000D2
:103EF00000000000000000000000000000000000C2
:103F000000000000000000000000000000000000B1
:0D3F100000000000000000000000000000A4
:020000040030CA
:0100000024DB
:010001000EF0
:010002003FBE
:010003001EDE
:010005008179
:010006008178
:010008000FE8
:01000900C036
:01000A000FE6
:01000B00E014
:01000C000FE4
:01000D0040B2
:00000001FF
